:100000000EC026C025C024C023C022C021C020C0ED
:100010001FC01EC01DC01CC061C01AC019C0112461
:100020001FBECFEDCDBF10E0A0E6B0E0ECE7F4E0FE
:1000300002C005900D92A036B107D9F710E0A0E6F6
:10004000B0E001C01D92A236B107E1F748D014C25A
:10005000D7CF0F931F93CF93DF938C0183EC81BD98
:10006000C0E0D0E013C0C29A000086B3C29882FDFF
:1000700005C0E0916000F0916100099585B780624C
:1000800085BF889585B78F7D85BF2196C017D1071D
:1000900050F3DF91CF911F910F910895282F80EC9D
:1000A00081BD90E008C085B7806285BF889585B71F
:1000B0008F7D85BF9F5F9217B0F30895282F83EC43
:1000C00081BD90E008C085B7806285BF889585B7FF
:1000D0008F7D85BF9F5F9217B0F308951895EF92BB
:1000E000FF920F931F93CF93DF9318BA17BA85B778
:1000F000877E806185BF789483EC81BD90E085B771
:10010000806285BF889585B78F7D85BF9F5F98305A
:10011000B1F734E060E070E0E3ECE1BD85B7806208
:1001200085BF889585B78F7D85BFC29A000026B3AD
:10013000C298822F90E0AC014470507022FD06C03E
:100140008FEF6F3F780711F06F5F7F4F832F322F54
:1001500082FDE3CF452B09F340E06530710508F4DB
:1001600041E0F4E056E0A3EC01C0FE2FA1BD85B74D
:10017000806285BF889585B78F7D85BFC29A000054
:10018000E6B3C2988E2F90E09C0124703070E2FD9F
:100190005150F2FD05C0232B19F04F5F56E0E5CF1B
:1001A000552319F783EC81BD90E085B7806285BF48
:1001B000889585B78F7D85BF9F5F9A30B1F74423BF
:1001C000D1F483EC81BD85B7806285BF889585B702
:1001D0008F7D85BF85B7806285BF889585B78F7D08
:1001E00085BFEB012297B89A82E090E032DFB898A1
:1001F000CE012FDFF8CF413021F4B89A84E090E0AF
:10020000BDC0423009F05FC0B89A80EC81BD85B7AF
:10021000806285BF889585B78F7D85BF85B78062F1
:1002200085BF889585B78F7D85BFB89880E190E0C0
:1002300010DFB89A80EC81BD90E085B7806285BF01
:10024000889585B78F7D85BF9F5F9330B1F7B8984C
:1002500080E190E0FEDEB89A80EC81BD90E085B749
:10026000806285BF889585B78F7D85BF9F5F9630FB
:10027000B1F7B89880E190E0ECDEB89A80EC81BDEF
:1002800090E085B7806285BF889585B78F7D85BFF3
:100290009F5F9131B1F7B89880E190E0DADEB89ACB
:1002A00088E090E0D6DEB89880E190E0D2DEB89A9F
:1002B00080E290E0CEDEB89880E190E0CADEB89AA5
:1002C00080E890E05BC0433009F068C080E190E0D6
:1002D000C0DEB89A81E090E0BCDEB89888E090E09B
:1002E000B8DEB89A80EC81BD90E085B7806285BFAA
:1002F000889585B78F7D85BF9F5F9630B1F7B89899
:1003000080E190E0A6DEB89A81E090E0A2DEB898A5
:1003100088E090E09EDEB89A84E090E09ADEB8989B
:1003200080E190E096DEB89A81E090E092DEB898A5
:1003300088E090E08EDEB89A80E190E08ADEB8989E
:1003400080E190E086DEB89A81E090E082DEB898A5
:1003500088E090E07EDEB89A80E490E07ADEB8989B
:1003600080E190E076DEB89A81E090E072DEB898A5
:1003700088E090E06EDEB89A8FEF90E06ADEB89881
:10038000E0916000F0916100099580E090E0DF91DC
:10039000CF911F910F91FF90EF900895443029F471
:1003A000B89A8FEF90E055DEFCCF93ECE92E80EC0D
:1003B000F82EC42FD0E02597B89AE1BC85B78062AB
:1003C00085BF889585B78F7D85BF85B7806285BFDE
:1003D000889585B78F7D85BFB89810E085B7806216
:1003E00085BF889585B78F7D85BFC29A000086B38B
:1003F000C29882FD05C0E0916000F091610009950E
:100400001F5F153059F7F1BC90E085B7806285BF5A
:10041000889585B78F7D85BF9F5F9530B1F700E0E8
:1004200024C0E1BC10E0C29A000086B3C29882FDED
:1004300005C0E0916000F0916100099585B7806288
:1004400085BF889585B78F7D85BF1F5F173059F7AA
:10045000F1BC90E085B7806285BF889585B78F7DB8
:1004600085BF9F5F9630B1F70F5F802F90E08C17AC
:0C0470009D070CF0A1CFD5CFF894FFCF72
:00000001FF
